:1000000002308A00432A0000D422532AA0264F2A15
:100010004F2955050000CC22D62CA0264F2A4F2967
:1000200020224F28D222C42A0A00D22C4324CC27D3
:10003000532A3A10A53A0A00D22C4324CC27532A3B
:100040003A10A53A0A00CC22D62CA0264F2A4F29D6
:1000500020224F2D412255050001D22C4324CC27CC
:10006000532A3A10A53A0A00D22C4324CC27532A0B
:100070003A10A53A0A005029412B5910CD27D42710
:100080005210C4275029452255050001D22C432483
:10009000CC27532A3A10A53A0A00D22C4324CC2765
:1000A000532A3A10A53A0A005029412B5910CD275E
:1000B000D4275210C427DA20C42A0A00D22C4324A1
:1000C000CC27532A3A10A53A0A00D22C4324CC2735
:1000D000532A3A10A53A0A00CB27CE224310D42245
:1000E000532A5510CD27D427D22A20270000CC220E
:1000F000D6203A10A53AA00400015029412B411DF9
:10010000A01275100900CC2FCE20D2205A1DA012AB
:1001100075100900D02FCE20D2205A1DA0127510C4
:100120000A00D027D72252104F2720050001CF25E3
:1001300021100A00D62C4229412AA0264F222E1730
:100140002E100A0083168613831286130830F800D7
:10015000A9280000F817BE28F81383160317930C7C
:100160008312031303188617031C86137817BE28FF
:100170007813F80BAD28BC28000086178430840063
:10018000840BC028C3280000F81BAC28781BB828B3
:100190000800831603178C170C140000000083124C
:1001A0000C087F39031915298316900083120D0856
:1001B0008316910083120F08831692001008930093
:1001C00083120313A22083160317110883128D00D4
:1001D0008316120883128F0083168C170C140000EC
:1001E000000083120C0D0E0D7F390319152983169B
:1001F000900083120D088316910083120F08831656
:1002000092001008930083120313A2208316031791
:10021000110883128D008316120883128F008D0A35
:1002200003198F0A0313C928031703130800831641
:1002300008108312081083168810831288109B01FF
:100240008A110A12432B8316081183120811831690
:1002500088118312881195018A110A12442B831682
:100260000317910111081002031C442937290313B5
:100270008812831288163C298316881283128812EA
:1002800083160317910A32298312031308004829A1
:1002900083168812831288164D29831688128312BA
:1002A00088120800013083160317930090309200E3
:1002B00003130812831208124721831603179301B0
:1002C00092019308031D84291208073C031C84290A
:1002D0001008120784008313111883170008940074
:1002E000140B792903130812831208167D2983162B
:1002F00003170313081283120812472183160317EA
:10030000920A0319930A612903130812831208162B
:1003100047210800831608128312081283168812D8
:10032000831288121E308316031790008312031362
:100330002F2183160812831208160A30831603171A
:100340009000831203132F2183160317910120308D
:100350009000831203135221053083160317900077
:10036000831203132F218316031791012830900065
:10037000831203135221831603179101303090002A
:100380008312031352218A110A12452B0830831657
:1003900003179702031CD829973084008317031092
:1003A000800C00080319D829D6290000800BD52914
:1003B000831203130800831603171308950012080D
:1003C00094009408031DE72995080319282A0313AC
:1003D000061283120616831686128312861283165D
:1003E000031711089600960A96030319FF29FF3098
:1003F000970083120313C62183160317F4291008EC
:10040000970083120313C621831686128312861661
:10041000831606128312061283160317110896001C
:10042000960A960303191C2AFF30970083120313C0
:10043000C62183160317112A10089700831203138D
:10044000C621831603171408031995039403E129A1
:10045000031383128A110A12512B913084008317DF
:1004600000080319402A0230F800F701F70B362A7A
:10047000F80B352A9730F700F70B3C2A800B332A0C
:100480008A110A12612B840183131F308305713096
:1004900083168F000F08861383128617831603179F
:1004A0000908C039890003131F129F120030031777
:1004B0008800831287018801890101300313A0009D
:1004C000A100A201A300A400A501A601A701A80004
:1004D000A900AA00AB00AC00AD01AE00AF01B001B5
:1004E000B101B201B301B401B501B601B7010317FF
:1004F0009001910192019301940195019601970158
:10050000980199019A019B019C019D019E019F0107
:10051000A001A101A201A301A401A501A601A701B7
:10052000A801A901AA01AB01AC01AD01AE01AF0167
:10053000B001B101B201B301B401B501B601B70117
:10054000B801B901BA01BB01BC01BD01BE01BF01C7
:10055000C001C101C201C301C401C501C601C70177
:10056000C801C901CA01CB01CC01CD01CE01CF0127
:10057000D001D101D201D301D401D501D601D701D7
:10058000D801D901DA01DB01DC01DD01DE01DF0187
:10059000E001E101E201E301E401E501E601E70137
:1005A000E801E901EA01EB01EC01ED01EE01EF01E7
:1005B000FF300313BA00913003178D0000308F0015
:1005C0000313C920831603170908C039FF388900AF
:1005D00003131F169F16FB300317880083120313A3
:1005E0001F179F1783169F1383121F149412BA129A
:1005F0003A088316870083123A163A088316870052
:100600008312BA113A0883168700013083129400CE
:100610000030831694000108C7390838810083121E
:1006200090010030F80006389200FF3083169200E7
:1006300083123A113A088316870083120711831632
:1006400009130C308312970083169B019C01013023
:100650009D008312BA103A08831687008312871010
:100660000C309D000130800003178701880189014B
:10067000831603139701051283120516831685123C
:1006800083128516172923298A2901308316031717
:100690009100F43090009301C8309200831203134C
:1006A000DB29973003178D0000308F000313C9201A
:1006B0000230831603179000FA309100831203135F
:1006C0002D2A83160317900B5C2B9A3083128D0012
:0C06D00000308F000313C9206C2B630066
:04400E00F52CFF3F4F
:00000001FF
